:020000040000FA
:020000001028C6
:08000800AA298207C034F93473
:10001000A434B034993492348234F8348034903437
:1000200003138312850107309F008316203085005B
:1000300000308600883081000C1083128B12013052
:1000400090001F3085000B178B17D101D201D3010F
:10005000D501D401C92068210E215418B92852189D
:1000600040285219482853185428851A63285214D6
:10007000473081000930D600C430D7008B162C28B9
:10008000D21C2C28D201851A2C2852154B212C2841
:10009000851E2C28D2015314473081000930D60028
:1000A000C430D7008B162C28D31C2C28851E2C2856
:1000B000D301CD0A0319CC0ACF0A0319CE0ADE20D8
:1000C0000E2152212C28BD200730500503192C2861
:1000D000D01C9228D01D2C2851187428CC01CD0199
:1000E000DE200E215D21B02855144730810061309B
:1000F000D600A830D7008B160E21D51C7C28BD2039
:10010000D01C9028D01D90280E2155197F285515F8
:10011000CE01CF01CC01CD01DE200E2164217F284C
:10012000D501B028501DAA28D01D2C284F084E04F8
:1001300003192C280130CF02031CCE034D084C04B8
:100140000319A6280130CD02031CCC03DE200E21AA
:100150005621B028501C2C280130D1060E214421F4
:100160005414473081000430D600E230D7008B169B
:100170002C28D41C2C28D4012C2883160F30860060
:10018000831206080F390F3AD000831686018312B6
:10019000080083169B011C141A089B078312C900D0
:1001A0004A3084000630DB0083169B0A1C141A08B0
:1001B00083128000840ADB0BD428080083169B017D
:1001C0008312CB0A031DF528CA0A031DF528063041
:1001D000C907490883169A001C1555309D00AA309E
:1001E0009D009C149C18F2288312490883169B07D3
:1001F00083124A3084000630DB00000883169B0A15
:100200009A001C1555309D00AA309D009C149C1826
:1002100007298312840ADB0BFD2808004E08511CB5
:100220004C08C0004F08511C4D08C100DC21FF30B4
:1002300086000514EF30511CDF3086000512922134
:10024000FF3086000516430805208600851192219F
:10025000FF3086008515440805208600051192218F
:10026000FF3086000515450805208600851092217F
:10027000FF3086008514460805208600051092216F
:10028000FF30860005140800FB30D8000430D90088
:1002900064308A210800FC30D8004430D900643032
:1002A0008A2108004421A4214B210800F830D800FD
:1002B0008930D90064308A210800F830D8008930AC
:1002C000D900FA308A2108005621A8215D210800B2
:1002D000F830D8008930D900C8308A21A621FA30F8
:1002E000D8001330D900C8308A21A621FB30D800AD
:1002F0000430D900C8308A21A621FC30D80044300F
:10030000D900C8308A21FC30D8004430D900C83028
:100310008A21080083160C148312972183160C106F
:10032000831208006430DE00DE0B94290800DD0033
:100330006E30DC009B299C299D29DC0B9A29A02981
:10034000A129DD0B982908001E3097293230972902
:1003500064309729F0000308F10083120B19B329C8
:100360000C18D029D7290B11473081000130D70252
:100370000319BE290318D729D602D729D608031D89
:10038000D729521CC529D214CE29531CC929D314EC
:10039000CE29541CCD29D414CE29D5148B12D7299B
:1003A0000C1058088F0059088E008030860671089E
:1003B0008300F00E700E090047308400E421E42130
:1003C000E421E421E42108001030C700C801031033
:1003D000C10DC00DC80DF63048070318C80003183A
:0E03E000C10AC70BE729840348088000080003
:02400E00023F6F
:0E4200000000000000000000000000000000B0
:1042C00043006F00700079007200690067006800A9
:1042D0007400200028004300290020003200300034
:1042E0003100380020006200790020004D002E00CF
:1042F000590061006D0061006D006F0074006F0077
:00000001FF
